:1000000008308A006E290000FF00030E8301A6005D
:100010007F08A5000A08AD008A01A50E0408A70004
:100020002008A8002108A9002208AA002308AB0084
:100030002408AC00831383128C308400801E222895
:100040008C1A3B288C308400801C28288C183D2872
:10005000270884002808A0002908A1002A08A20077
:100060002B08A3002C08A4002D088A00260E83006C
:10007000FF0E7F0E09008A113C2B8A11512C0A10A9
:100080008A100A118207203420344E34433400345D
:100090000A108A100A11820720344534523452342F
:1000A00000340A108A100A11820720344F34763443
:1000B000653472342034743465346D3470340034F3
:1000C0000A108A100A11820761346C346134723468
:1000D0006D347334203465346E34613462346C347E
:1000E000653464343A3400340A108A100A118207E5
:1000F00031343A3420342534303434346C3475346B
:10010000203432343A3420342534303434346C34AE
:10011000753400340A108A100A11820733343A34D5
:1001200020342534303434346C3475342034343451
:100130003A3420342534303434346C34753400345B
:100140000A108A100A118207443465346734203457
:10015000463461346834723465346E3468346534DE
:100160006934743400340A108A100A118207443446
:10017000653467342034433465346C347334693403
:100180007534733400340A108A100A1182074D3412
:100190006134783400340A108A100A11820720343E
:1001A0004D346134783400340A108A100A11820701
:1001B00020344D3469346E347334203461346E34F9
:1001C000643420344D34613478346534733400340D
:1001D0000A108A100A118207203420342034203477
:1001E00020345234653473346534743400340A1066
:1001F0008A100A1182074D3469346E3400340A14AF
:100200008A100A11820720344D3469346E34003468
:100210000A148A100A11820731343A342034003427
:100220000A148A100A118207203432343A342034F6
:1002300000340A148A100A11820733343A34203405
:1002400000340A148A100A118207203434343A34F4
:10025000203400340A148A100A1182070D340A343B
:100260002334203428342534643429340D340A34BA
:1002700000340A148A100A118207233420345434BB
:100280006834653472346D346F346B342034283400
:1002900063342934203441345034523453342034BC
:1002A00057346F3472346C3464342C3420344C340E
:1002B0004C3443342034253473340D340A34003440
:1002C0000A148A100A118207323430342D3446342D
:1002D000653462342D343034373400340A148A10D3
:1002E0000A1182072334203468347434743470342F
:1002F0003A342F342F347734773477342E346134D2
:1003000070347234733477346F3472346C346434D0
:100310002E3463346F346D342F3474346834653460
:1003200072346D346F346B342F340D340A3400342E
:100330000A148A100A1182072334203475346E346B
:100340006934743473343D34253455342034613485
:100350006C34613472346D345F34613463347434BA
:100360006934763465345F3473347434613474348E
:1003700065343D34253455340D340A3400340A14C0
:100380008A100A1182072334203441342034613426
:100390006C34613472346D342034733465347434A5
:1003A000203470346F3469346E34743473343A34B6
:1003B000203425346C347534203425346C34753451
:1003C000203425346C347534203425346C34753441
:1003D0000D340A3400340A148A100A11F23E03184C
:1003E0008A0A8200233420344234203461346C344D
:1003F000613472346D342034733465347434203491
:1004000070346F3469346E34743473343A34203455
:1004100025346C347534203425346C3475342034F0
:1004200025346C347534203425346C3475340D34F3
:100430000A3400340A108A140A1182072334203443
:1004400061346C34613472346D342034413420347E
:100450006F346E342034253455342034623465349E
:1004600063346134753473346534203425346C342A
:10047000753420343E34203425346C3475342C34B7
:100480002034733465347434743469346E346734AE
:1004900020344134203474346F34203425345534BE
:1004A0000D340A3400340A108A140A1182072334E6
:1004B000203461346C34613472346D34203442340D
:1004C00020346F346E342034253455342034623473
:1004D00065346334613475347334653420342534C1
:1004E0006C34753420343E34203425346C34753407
:1004F0002C342034733465347434743469346E3479
:10050000673420344234203474346F34203425343A
:1005100055340D340A340034831626088312A101A1
:10052000831625020318992A25088312A000AC2AF5
:1005300083168312A00108308316A700A50D83122D
:10054000A00D83162608831220020318A000A10D17
:100550008316A70B9E2A8312003420308316201E98
:100560003030A10083127E08A000FE1FC02AA0091F
:10057000A00A2008FE002D308316A100A0178312C8
:100580007E088316A5006430A60083128C22200802
:10059000FE00303021078316A20083127E088316E6
:1005A000A5000A30A60083128C2230302007831663
:1005B000A4003030831221078316A3002108831280
:1005C000A0008316A01DE62AA01F2011201AF72ADA
:1005D000A01F162B2019162B831220088316A200A9
:1005E000A018162B831220088316A300162B303078
:1005F0002202031D162B831220088316A20020302E
:10060000A100A01D072B2011A014A01FA0103030A6
:100610002302031D162B831220088316A30020300B
:10062000A200A01D072BA010A01F2010201D202B12
:10063000210883120C1A1E2B8316192B990083167E
:10064000A01C2A2B220883120C1A282B8316232B7A
:1006500099008316201C342B230883120C1A322B8A
:1006600083162D2B99008316240883120C1A3A2B1B
:100670008316352B990000348C1E3C2B1A08FB0086
:100680007B080C1E412B99007B08403C03184F2B24
:100690007B085A3C031C4F2B7B082038502B7B08CF
:1006A000FB007B08663A03195F2B123A0319842B6F
:1006B000193A0319A82B083A0319E92B2B2C0130FE
:1006C000B7000430FC00FD017D082A21FD0AA000CE
:1006D00020080C1E692B990005307D02031D642B38
:1006E0007C08FE001F308316A0008312AD22293043
:1006F0000C1E782B99000D300C1E7C2B99000A30B3
:100700000C1E802B99004E2CB7010530FC00FD011A
:100710007D082A21FD0AA00020080C1E8D2B9900BF
:1007200005307D02031D882B7C08FE001F308316D8
:10073000A0008312AD2229300C1E9C2B99000D3095
:100740000C1EA02B99000A300C1EA42B99004E2CD5
:10075000B501213003178D000313350803178C00F2
:1007600083168C130C15831203130B08A0008B1334
:100770008316031755308D00AA308D008C148C1809
:10078000BF2B0C118312031320088B040630FC00CE
:10079000FD017D082A21FD0AA00020080C1ECE2B99
:1007A000990005307D02031DC92B7C08FE001F3017
:1007B0008316A0008312AD2229300C1EDD2B990078
:1007C0000D300C1EE12B99000A300C1EE52B990010
:1007D0004E2C0130B500213003178D00031335086E
:1007E00003178C0083168C130C15831203130B084C
:1007F000A0008B138316031755308D00AA308D008F
:100800008C148C18012C0C118312031320088B04F8
:100810000730FC00FD017D082A21FD0AA000200808
:100820000C1E102C990005307D02031D0B2C7C083A
:10083000FE001F308316A0008312AD2229300C1E4B
:100840001F2C99000D300C1E232C99000A300C1E11
:10085000272C99004E2C0130FC00FD017D082A2137
:10086000FD0AA00020080C1E332C990005307D02E3
:10087000031D2E2C7C08FE001F308316A00083125F
:10088000AD2229300C1E422C99000D300C1E462C36
:1008900099000A300C1E4A2C99004E2C8C128A1199
:1008A0002828E408031D5D2CE508031D5D2CE501E7
:1008B0006430E4000130B900612C64080319E503D9
:1008C000E403831606140030831206180130003A40
:1008D000031D732C380B6D2C732C0130B8000330C2
:1008E000E300E830E2006208630403197B2C62082D
:1008F0000319E303E203E208031D822CE308031D4E
:10090000822CB8018C108A1128286B3084000008D2
:100910000319992C0130A100A001A00B8D2CA10B73
:100920008C2C4A30A000A00B932C00000000800B00
:100930008A2C00348316861183128615831686113D
:10094000831286110034FA1BA72C8510A82C85145D
:100950008316851083127A1BAF2C0510B02C05145A
:10096000831605108312FA1AB72C8612B82C861635
:100970008316861283127A1ABF2C0612C02C061612
:100980008316061283129A24FA19C82C8510C92CD2
:1009900085148316851083127A19D02C0510D12C5A
:1009A0000514831605108312FA18D82C8612D92C38
:1009B00086168316861283127A18E02C0612E12C12
:1009C00006168316061283129A240D30A000A00B7F
:1009D000E72C00340030A10005389200F93083166E
:1009E00092008C148C160F308312EB008524831632
:1009F0008610831286108316061183120611831641
:100A00008510831285108316051083120510831636
:100A100086128312861683160612831206169A24ED
:100A20000530EB0085249A242130A000A00B162D60
:100A30009A240530EB0085248316061283120612D1
:100A40009A240D30A000A00B232D2830FA00A324F7
:100A50000C30FA00A3240630FA00A3240130FA0077
:100A6000A324B41234088316870083128716341126
:100A70003408831687008312071534103408831650
:100A8000870083120714B41034088316870083127A
:100A90008714B411340883168700831287118A15CE
:100AA00094296F08FC3E0318862D043E872DF0081C
:100AB000031D5C2D87105D2D8714B4103408831638
:100AC00087008312862DF008031D682D0710692DFD
:100AD000071434103408831687008312862DF0081B
:100AE000031D742D0711752D071534113408831655
:100AF00087008312862DF008031D802D8712812D1B
:100B00008716B412340883168700831200340A143F
:100B10008A100A158207572D632D6F2D7B2DEC014E
:100B2000ED016B08EF00F00151250630A000A00B8D
:100B3000972D0000EE016E080F3C031CC32DB4116D
:100B4000340883168700831287151030A000A00B8D
:100B5000A72D000034163408831687008312071A65
:100B6000B32D0310B42D0314EC0DED0DB4113408A6
:100B700083168700831287111030A000A00BBE2DB2
:100B80000000EE0A9B2D6B08EF000130F0005125AC
:100B90006C08A1006D08A2000034E7016708033C5F
:100BA000031CEB2D6708EB008F250310670D3A3E01
:100BB0008400840A2730800084030F3080000310F3
:100BC000670D423E8400840A2730800084030F3082
:100BD0008000E70ACE2D003483168610831286101B
:100BE0000130FA00A3240230EB0085240034831680
:100BF00086108312861080306A07EB00FA00A32467
:100C0000003483168610831286147908FA00A32410
:100C100000340408F800720EF038F400F407E23EE5
:100C2000F500323EF70072080F39F507F507F707B0
:100C3000E93EF600F607F607710E0F39F607F707DB
:100C4000F60DF70DF709F70D71080F39F707F40DD9
:100C50000730F3000A30F707F603031C2B2EF607C4
:100C6000F503031C2F2EF507F403031C332EF407A2
:100C7000F303031C372E7330840007307805781394
:100C8000840777300402031978170008A000031DB9
:100C9000512E781B512E781A5D2EF819512E2030C6
:100CA000542EF81578123030A007F2010408F10034
:100CB0002008F900012671088400840A781F412E5B
:100CC0000034E808031D672E4130E900692E4230E8
:100CD000E9000310680D523E8400840A0008A30056
:100CE00084030008031DAD2EA308031DAD2E0130A3
:100CF0006807A0000310A00D2008523E8400840A5B
:100D00000008A30084030008031DAD2EA308031DE3
:100D1000AD2E02306807A0000310A00D2008523E3F
:100D20008400840A0008A30084030008031DAD2E7C
:100D3000A308031DAD2E03306807A0000310A00D0B
:100D40002008523E8400840A0008A300840300089F
:100D5000031DAD2EA3080319582FEC25EA01F72532
:100D60006908F9000126EA016A08512000380319D0
:100D7000BD2EEA0AF9000126B42E4030EA00F7251C
:100D8000EA016A08602000380319CA2EEA0AF9004D
:100D90000126C12E0630EA00FA30EB008524EA0B6A
:100DA000CC2EEC25EA01F7250310680D523E840095
:100DB000840A0008EB0084030008EA000130680799
:100DC000A0000310A00D2008523E8400840A0008F1
:100DD000EE0084030008ED003130F90001263A30BE
:100DE000F90001262030F9000126093084006B0843
:100DF000F2006A08F10009260830EF006F0874203D
:100E0000EF0AA000F90001260C306F02031DFE2E30
:100E1000093084006E08F2006D08F10009264030A8
:100E2000EA00F72502306807A0000310A00D200893
:100E3000523E8400840A0008EC0084030008EB00A2
:100E400003306807A0000310A00D2008523E840064
:100E5000840A0008EF0084030008EE003330F90034
:100E600001263A30F90001262030F9000126093028
:100E700084006C08F2006B08F10009260830F000CD
:100E800070088A20F00AA000F90001260C307002D8
:100E9000031D402F093084006F08F2006E08F10036
:100EA00009260630EA00FA30EB008524EA0B532FBE
:100EB00000342108AE018B1BAE178B136F0883160D
:100EC000A5006430A60083128C22AE1B8B1720086D
:100ED000EF0021083030031D742FF01C7C2FF01917
:100EE0007C2F701A2030772FF01170127014A10728
:100EF00021080C1E792F9900AE018B1BAE178B13A6
:100F00006F088316A5000A30A60083128C22AE1B40
:100F10008B172008EF0021083030031D952FF019A2
:100F20009A2F701C9A2F701A2030A10721080C1ECE
:100F3000972F99003030EF076F080C1E9D2F9900F6
:100F400000340408F5006F0EF038F100F107E23EBE
:100F5000F200323EF4006F080F39F207F207F4078F
:100F6000E93EF300F307F3076E0E0F39F307F407BA
:100F7000F30DF40DF409F40D6E080F39F407F10DBB
:100F80000730F0000A30F407F303031CC32FF30704
:100F9000F203031CC72FF207F103031CCB2FF10749
:100FA000F003031CCF2F70308400073075057513D4
:100FB000840774300402031975170008A000031D8C
:100FC000E92F751BE92F751AF12FF519E92F20303C
:100FD000EC2FF51575123030A00720080C1EEE2FEF
:0A0FE0009900840A751FD92F003410
:101000006A10E7016708033C031C9D286708EB0092
:101010008A118F258A152208E9002108E80000308E
:1010200068190130013C031D17286A1418286A103A
:10103000E90CE80CE90CE80CE90CE80CE90CE80C0C
:10104000E90CE80C0730E9056A1854280310670D0D
:101050003A3E8400840A0008A30084030008A1002B
:1010600023086902031C3A28031D4A286808210244
:10107000031C4A280310670D3A3E8400840A0008C6
:10108000A300840300080F3C031D54282308273CB9
:10109000031D54280310670D3A3E8400840A690832
:1010A00080008403680880006A1884280310670D94
:1010B000423E8400840A0008A30084030008A100C3
:1010C00069082302031C6A28031D7A282108680284
:1010D000031C7A280310670D423E8400840A00082E
:1010E000A300840300080F3C031D84282308273C29
:1010F000031D84280310670D423E8400840A69089A
:1011000080008403680880006A1891280310670D26
:101110004A3E8400840A69088000840368088000CD
:101120009B280310670D4A3E8400840A2730800004
:1011300084030F308000E70A02288A15DB2B093070
:1011400084004B08EF004A08EE008A11A1278A1597
:1011500020300C1EA9289900093084004D08EF00AA
:101160004C08EE008A11A1278A1520300C1EB628E3
:101170009900093084004F08EF004E08EE008A11F4
:10118000A1278A1520300C1EC3289900093084003D
:101190005108EF005008EE008A11A1278A150D3082
:1011A0000C1ED02899000A300C1ED42899008A15EC
:1011B000672D1030ED00A001A301EA0CE90C031C1F
:1011C000E7286B08A0070318A30A6C08A307A30C61
:1011D000A00CA20CA10CED0BDD288A155129A10150
:1011E000A201A001A3016E08031DF9286D080319CF
:1011F00013291030EF000310EB0DEC0DA00DA30D23
:101200006E082302031D06296D082002031C0F2906
:101210006D08A002031CA3036E08A3020314A10D12
:10122000A20DEF0BFB2800008A155D2967080F3C13
:10123000031D2D296808273C031D2D29E901690894
:101240008A113F208A15003803192C29E90AF90070
:101250008A1101268A151F296D296808063C031882
:101260004729FF3A031D382967086C3C03184729B2
:10127000E90169088A1148208A15003803194629AE
:10128000E90AF9008A1101268A1539296D29350BD9
:1012900064296808EA006708E900EC010930EB00FE
:1012A000D9282208EA002108E9002208EC002108D8
:1012B000EB00EE010530ED00EF2820302107E700BC
:1012C0002208E8000318E80A013084006808F200E8
:1012D0006708F1008A1109268A15003484011F303D
:1012E00083051930831699002630980090308312B8
:1012F000980083161F149F141F159F1107309C0020
:101300008312AF010130B000B101B201B301FF306F
:10131000B400B501B601B701B801B901E201E301BA
:10132000E401E5018A11EA2C8A15323003178D0099
:1013300083168C130C1483120C080313B6003608A2
:10134000013C0318C129B601323003178D00031385
:10135000360803178C0083168C130C1583120313A5
:101360000B08A0008B138316031755308D00AA308D
:101370008D008C148C18BA290C11831203132008C9
:101380008B04213003178D0083168C130C148312E9
:101390000C080313B5003508013C0318ED29B5010D
:1013A000213003178D000313350803178C008316B3
:1013B0008C130C15831203130B08A0008B138316D8
:1013C000031755308D00AA308D008C148C18E62937
:1013D0000C118312031320088B04831606140030AB
:1013E000831206180130003A031D1A2AB5080319A2
:1013F000FB290030FC290130B500213003178D0096
:101400000313350803178C0083168C130C158312F5
:1014100003130B08A0008B138316031755308D00A0
:10142000AA308D008C148C18132A0C11831203130C
:1014300020088B04E7016708073C031C4F2A0310B0
:10144000670D523EE8000310670D223EE90069086F
:10145000EA006A0803178D0083168C130C1483129C
:101460000C080313EB0001306A07ED0003178D0031
:1014700083168C130C1483120C080313EC006B08F6
:10148000A3006C08A1006B08A20068088400840A0D
:1014900022088000840321088000E70A1B2A8316A3
:1014A00085118312851583168512831285168A117C
:1014B000CD258A158A11EC258A15B608031D622AE6
:1014C0008511632A8515831685118312B608031DBD
:1014D0006B2A85126C2A8516831685128312EA01FF
:1014E0008A11F7258A15E70167080F3C031C962A25
:1014F000670803178D0083168C130C1483120C08D5
:10150000031D852A0313962A03170313670803177D
:101510008D0083168C130C1483120C080313E8003F
:10152000F9008A1101268A15E70A742A4030EA0078
:101530008A11F7258A15350BAC2AE80168088A114B
:10154000A0208A1500380319AB2AE80AF9008A118D
:1015500001268A159E2ABA2AE80168088A11B32052
:101560008A1500380319BA2AE80AF9008A110126F7
:101570008A15AD2A0630E800FA30EB008A1185247E
:101580008A15E80BBC2AE8018A1161268A15043005
:10159000E8008A1161268A15B6080319D12A851137
:1015A000D22A8515831685118312B6080319DA2A03
:1015B0008512DB2A8516831685128312E7016708D8
:1015C0008A1139218A15E70AA00020080C1EE62A94
:1015D00099001E306702031DDF2AE80168088A119E
:1015E00060218A1500380319FA2AE80A0C1EF62A27
:1015F0009900EE2A0D300C1EFB2A99000A300C1EB1
:10160000FF2A9900E70167088A116E218A150038C0
:1016100003190F2BE70A0C1E0B2B9900032BE70174
:1016200067088A1198218A15E70AA00020080C1E75
:10163000172B990008306702031D102B3508EF00A7
:101640001B30F0008A1159278A150A30E800680813
:101650008A1198218A15E80AA00020080C1E2E2B5A
:1016600099001E306802031D272B3608EF001B303F
:10167000F0008A1159278A150D300C1E3D2B990058
:101680000A300C1E412B9900E70167088A11BF211F
:101690008A15E70AA00020080C1E4C2B9900163072
:1016A0006702031D452B103084005308EF005208D9
:1016B000EE008A11A1278A1520300C1E5D2B99009F
:1016C000103084005508EF005408EE008A11A1275D
:1016D0008A1520300C1E6A2B9900103084005708A0
:1016E000EF005608EE008A11A1278A1520300C1E43
:1016F000772B9900103084005908EF005808EE004D
:101700008A11A1278A150D300C1E842B99000A30EE
:101710000C1E882B9900E70167088A11EB218A15B6
:10172000E70AA00020080C1E932B990016306702D0
:10173000031D8C2B103084005B08EF005A08EE006C
:101740008A11A1278A1520300C1EA42B9900103075
:1017500084005D08EF005C08EE008A11A1278A155D
:1017600020300C1EB12B9900103084005F08EF0070
:101770005E08EE008A11A1278A1520300C1EBE2BB0
:101780009900103084006108EF006008EE008A11B3
:10179000A1278A150D300C1ECB2B99000A300C1E88
:1017A000CF2B9900C0308B048A11EC258A15B9081B
:1017B0000319682D0028E6016608033C031C9B2CD6
:1017C0000310660D4A3E8400840A0008E800840382
:1017D0000008E7000F3C031DF12B6808273C0319A4
:1017E000902C0310660D4A3E8400840A0008EA002B
:1017F00084030008E9000310660D523E8400840A49
:101800000008A30084030008A10023086A02031C47
:10181000902C031D0F2C690821020318902C031033
:10182000660D4A3E8400840A0008E800840300082C
:10183000E7000310660D523E8400840A0008EA00A7
:1018400084030008E900EB016B088A111A228A154B
:10185000EB0AA00020080C1E2B2C99000D306B0207
:10186000031D242C6608EF001B30F0008A11592755
:101870008A150F30EC006C088A111A228A15EC0ABE
:10188000A00020080C1E422C990018306C02031D89
:101890003B2C103084006808EF006708EE008A11C6
:1018A000A1278A1520300C1E532C99003E300C1EA7
:1018B000572C990020300C1E5B2C990010308400AE
:1018C0006A08EF006908EE008A11A1278A15213005
:1018D000ED006D088A111A228A15ED0AA000200871
:1018E0000C1E702C990030306D02031D692C3608D7
:1018F000EF001B30F0008A1159278A150D300C1E9D
:101900007F2C99000A300C1E832C9900B608031D09
:101910008B2C85118C2C851583168511982C8312A0
:10192000B6080319952C8511962C851583168511FB
:101930008312E60ADC2BE6016608033C031C632DD8
:101940000310660D4A3E8400840A0008E800840300
:101950000008E7000F3C031DB12C6808273C031961
:10196000582D0310660D4A3E8400840A0008EA00E0
:1019700084030008E90004306607A0000310A00DEE
:101980002008523E8400840A0008A3008403000853
:10199000A10023086A02031C582D031DD32C6908DB
:1019A00021020318582D0310660D4A3E8400840A54
:1019B0000008E80084030008E70004306607A00080
:1019C0000310A00D2008523E8400840A0008EB009A
:1019D00084030008EA00EC016C088A1153228A157E
:1019E000EC0AA00020080C1EF32C99000D306C02AC
:1019F000031DEC2C6608EF001B30F0008A115927FC
:101A00008A150F30ED006D088A1153228A15ED0AF0
:101A1000A00020080C1E0A2D990018306D02031D2D
:101A2000032D103084006808EF006708EE008A116B
:101A3000A1278A1520300C1E1B2D99003E300C1E4C
:101A40001F2D990020300C1E232D9900103084008A
:101A50006B08EF006A08EE008A11A1278A15213071
:101A6000EE006E088A1153228A15EE0AA0002008A3
:101A70000C1E382D990030306E02031D312D3608B2
:101A8000EF001B30F0008A1159278A150D300C1E0B
:101A9000472D99000A300C1E4B2D9900B608031DE6
:101AA000532D8512542D851683168512602D8312B1
:101AB000B60803195D2D85125E2D851683168512D5
:101AC0008312E60A9C2CB708031D672D9F28B901D5
:101AD000B808031DCA2DEA018A11F7258A15E70106
:101AE00067088A1108218A15003803197D2DE70A35
:101AF000F9008A1101268A15702D4B08E8004A0862
:101B0000E7001621E70167088A1110218A150038BD
:101B10000319902DE70AF9008A1101268A15832DF1
:101B20004D08E8004C08E70016214030EA008A1111
:101B3000F7258A15E70167088A1119218A150038E7
:101B40000319A82DE70AF9008A1101268A159B2D91
:101B50004F08E8004E08E7001621E70167088A11E0
:101B600021218A1500380319BB2DE70AF9008A11D3
:101B700001268A15AE2D5108E8005008E70016210D
:101B80000330E700C830EB008A1185248A15E70B83
:101B9000C22DCC2E380BCC2E8A11EC258A15EA01E9
:101BA0008A11F7258A15E70167088A11C3208A156B
:101BB00000380319E12DE70AF9008A1101268A1578
:101BC000D42D3B08E8003A08E7001621E701670832
:101BD0008A11CB208A1500380319F42DE70AF90081
:101BE0008A1101268A15E72D3D08E8003C08E70028
:101BF00016214030EA008A11F7258A15E7016708A7
:101C00008A11C3208A15003803190C2EE70AF9003F
:101C10008A1101268A15FF2D3F08E8003E08E700DB
:101C20001621E70167088A11CB208A1500380319AD
:101C30001F2EE70AF9008A1101268A15122E410883
:101C4000E8004008E70016210830E700FA30EB0012
:101C50008A1185248A15E70B262E83160614003078
:101C6000831206180130003A031D6B2E8A11CD2510
:101C70008A158A11EC258A15EA018A11F7258A1539
:101C8000E70167088A11D4208A15003803194E2EFF
:101C9000E70AF9008A1101268A15412E4030EA0030
:101CA0008A11F7258A15E70167088A11E8208A1545
:101CB00000380319612EE70AF9008A1101268A15F6
:101CC000542E0830E700FA30EB008A1185248A157B
:101CD000E70B632ECC2E8A11EC258A15EA018A11B6
:101CE000F7258A15E70167088A11F7208A15003859
:101CF0000319802EE70AF9008A1101268A15732E2E
:101D00004308E8004208E7001621E70167088A1146
:101D1000FF208A1500380319932EE70AF9008A116B
:101D200001268A15862E4508E8004408E70016219A
:101D30004030EA008A11F7258A15E70167088A1101
:101D4000F7208A1500380319AB2EE70AF9008A112B
:101D500001268A159E2E4708E8004608E70016214E
:101D6000E70167088A11FF208A1500380319BE2E83
:101D7000E70AF9008A1101268A15B12E4908E80000
:101D80004808E70016210830E700FA30EB008A1116
:0C1D900085248A15E70BC52ED72B6300B5
:021E00000034AC
:1042000054006800650072006D006F006B002000B4
:044210003200000078
:0242420000007A
:02400E00723FFF
:00000001FF
